:030000000211F6F4
:03000B000200BE32
:03002B00020400CC
:03005B0002054457
:0300730002053A49
:1000800002030406080C10182030406080020304AC
:1000900006080C101820304080FF0406080C1018C9
:1000A0002030406080A0C000000001010003020277
:1000B000010505020D0505050D0604050202C2AF86
:1000C000C0D0C0E0205A25302F02E47330601A05FA
:1000D00060C37405952540F2956040EE758A78E519
:1000E000257003758A000203F90203EC306306C22F
:1000F000B1C287C28185258AC25AE525F4700221E2
:10010000DF0561306013206A19758B00D0E0D0D014
:10011000C2B1C287C281D2AF32C2B1C287C281022C
:1001200001CFD26EC26FE565601CC3E561149565B1
:100130004014C26ED26FC3E561956450030201CFD3
:100140007561000201CF206C14C2B1C287C28174F4
:1001500006D5E0FDD282D286D2800201CFD26FC214
:10016000B1C287C281E53D20E23420E1127406D598
:10017000E0FD207502D280307502D2820201CF20CC
:10018000E0127406D5E0FD207502D280307502D2EF
:10019000820201CF7406D5E0FDD2860201CF20E1B4
:1001A0001F20E00A7406D5E0FDD2860201CF740656
:1001B000D5E0FD207502D282307502D2800201CFD7
:1001C0007406D5E0FD207502D282307502D28075AA
:1001D0008B00D0E0D0D0C2B1C287C281D2AF32D0C2
:1001E000E0D0D0D2AF3261ECE525600A207502D2B2
:1001F000B1307502D281C28761ECE5256002D287F9
:10020000207502C281307502C2B161ECE525600A39
:10021000207502D281307502D2B1207502C2B13090
:100220007502C28161EC207502C282307502C28003
:10023000E525600A207502D2B1307502D2812075A1
:1002400002C280307502C282C28761EC207502C290
:1002500082307502C280207502C280307502C2826F
:100260007406D5E0FDE525600A207502D2B130752F
:1002700002D281C28761EC207502C282307502C24F
:1002800080E525600A207502D2B1307502D281C2A4
:1002900086C28761EC207502C282307502C280C2BC
:1002A000867406D5E0FDE525600A207502D2B130DE
:1002B0007502D281C28761ECC286E5256002D287D1
:1002C000207502C282307502C280207502C2813060
:1002D0007502C2B161ECC286207502C2823075021D
:1002E000C2807406D5E0FDE5256002D28720750244
:1002F000C281307502C2B161ECC286E5256002D2CE
:1003000087207502C280307502C282207502C281C8
:10031000307502C2B161ECC286207502C2803075B0
:1003200002C2827406D5E0FDE5256002D287207501
:1003300002C281307502C2B161EC207502C2803008
:100340007502C282E525600A207502D281307502ED
:10035000D2B1C286207502C2B1307502C28161EC91
:10036000207502C280307502C282C2867406D5E052
:10037000FDE525600A207502D281307502D2B120D8
:100380007502C2B1307502C28161EC207502C28073
:10039000307502C282E525600A207502D28130756F
:1003A00002D2B1207502C282307502C2802075026D
:1003B000C2B1307502C28161EC207502C280307515
:1003C00002C282207502C282307502C2807406D5D4
:1003D000E0FDE525600A207502D281307502D2B1B8
:1003E000207502C2B1307502C28161ECE525F4F5D9
:1003F0008A758B00756000D25AD0E0D0D0D2AF326F
:10040000C2AFC0D0C0E0D2D3C2CEE528600A741F0C
:10041000552E60491528815D78007900E580307699
:1004200001F430E50278FF53DACF20760343DA2077
:1004300030760343DA10C2D8C269E580307601F421
:1004400030E50279FFC3E89970CE3059037528185A
:10045000741F552E60037528188858D268E52960E6
:100460000415298170741F552E600543DA01C2D826
:0E047000206802A102E558F8C268741F552EDC
:10047E0060367982B70431C3E894F0400374F0F823
:10048E00E8C4540F28F87984B7030281B6C313C3A6
:10049E00138721200802C313200A06C3C898F881C7
:1004AE00B628F8500374FFF8C3E8955F5003E55F74
:1004BE00F8E52C5406703D882230630AC3E5229578
:1004CE005C4003855C227882B60429C3E52295241C
:1004DE00401278A096400DE52426F5245009752487
:1004EE00FF0204F5852224852425C3E524955C406E
:1004FE0003855C2520CF09D0E0D0D0C2D3D2AF3255
:10050E00C2CF7801E5286008741F552E7002152899
:10051E00C3E55894014005755B00A131E55B0460AD
:10052E0002055BD0E0D0D0C2D3D2AF32C2AF53916E
:10053E007FC258D2AF32C2AFC0D0C0E0C0F0D2D36B
:10054E00A8FBA9FCC2D8306902A1A753DACF207646
:10055E000343DA1030760343DA20D269E580307631
:10056E0001F420E502A17B88268927E14753DACFE3
:10057E0020760343DA2030760343DA10C2D8C269FC
:10058E00741F552E7002E12D7800E580307601F44F
:10059E0030E502E12D8858E12D53DACF2076034362
:1005AE00DA2030760343DA10C269205902C1615352
:1005BE00DACF20760343DA1030760343DA20C2D83E
:1005CE00D26988538954C3E89551F8E99552F9E4F4
:1005DE00FB7AFAC3E894C8E994005008E4D2E4FB2D
:1005EE007A0AC134C3E89468E994015008E4D2E36E
:1005FE00FB7A0FC134C3E894D0E994025008E4D2D8
:10060E00E2FB7A1EC134C3E894A0E994055008E4D5
:10061E00D2E1FB7A3CC134C3E89498E994085006C1
:10062E00E4D2E0FB7A78C3E89555FCE99556FD30A7
:10063E00E708ECF42401FCEDF4FD7557007008C3D7
:10064E00EC9A500375570188558956A853A95488BA
:10065E00518952C3E89526F8E99527F9307402E1DD
:10066E0000307302E100307202C1F9E9C313F9E8F8
:10067E0013F8307102C1F9E9C313F9E813F83070B9
:10068E0002C1F9E9C313FDE813FC205918C3EC9419
:10069E001CED9402400302072DED7009C3EC94C8C3
:1006AE00500302074774002077037896E624FAFE7B
:1006BE00E43400FFC3EC9EFCED9FFD5006780079FC
:1006CE0000E100C3EC94FFED9400400678FF790042
:1006DE00E100EC856CF0A4C5F0A2F733F879004088
:1006EE000302071C78FF790002071CE9C313F9E81F
:1006FE0013F830740EE9600278FFC3E81338F8E49B
:10070E003400F9C3E894FFE99400400278FF88585A
:10071E00D268205902E12D741FF4552E4BF52E751B
:10072E002818741F552E700375280A305902E14798
:10073E00741F552E600353DAFE752906741F552E4D
:10074E00700375290AD0F0D0E0D0D0C2D3D2AF3228
:10075E007901E1767903E176790AE176791EE1761F
:10076E007964E17679C8E1767817E4D5E0FDD8FAB8
:10077E00D9F6227A147B7802079D7A107B8C0207B9
:10078E009D7A0D7BB402079D7A0B7BC802079DAC48
:10079E00257525017902B275E4C286D5E0FDE52501
:1007AE006002D287D5E0FDC287D5E0FDD286D5E0C6
:1007BE00FDE525600A207502D2B1307502D281E5C1
:1007CE006DD5E0FD207502C2B1307502C2817496FE
:1007DE00D5E0FDD9C1EAF8D5E0FDD8FBDBB1C28684
:1007EE008C2522C37C007D0075F00005F0EA33FAFB
:1007FE00EB33FB50F6EB13FBEA13FAC3E9FFE8FE0B
:10080E00E89AF8E99BF95004EFF9EEF8B3EC33FCF3
:10081E00ED33FDD5F0DFEDF9ECF822E889F08A2012
:10082E00D2D4F8A9F07B0030F70B7BFFF42401F84B
:10083E00E9F43400F9E88520F0A4ADF0F8E985205C
:10084E00F0A4AFF0FEED2EF974003FFA7C04C3EA7B
:10085E0013FAE913F9E813F8DCF48BF030F70AE831
:0F086E00F42401F8E9F43400F9E889F0C2D4F871
:10087D00A9F0227882B6040302090CC3E55894014D
:10088D004018E54870377805C37994B7020278129D
:10089D00C3E53B9400E53C984020E5486009855E42
:1008AD005D7562FF756301852224E4F53FF540F522
:1008BD0041F542F543F54802090C754801C3799499
:1008CD00E79402601BE523F43333F913F8E954017F
:1008DD0004F9E854FEC39440F8E99400F9020908BC
:1008ED00E523F433333333F913F8E954070404F9EA
:1008FD00E854F8C39440F8E99400F9883F89402200
:10090D00E548603BC3E53C13F9E53B13F8C3E53F10
:10091D0098F8E54099F9500CC3E89480E994FF40AC
:10092D0016020948C3E8947FE99400500302094870
:10093D00787F7900020948788079FF8844894522BB
:10094D00E5486058E5442541F8E5453542F98545CA
:10095D0020E4300701F43543FA30E709C3EA94F097
:10096D00401502098AC3EA940F500302098A78FFE1
:10097D0079FF7A0F02098A780079007AF0C3E524AD
:10098D00955C5006E524600921A3E54520E70D217E
:10099D00A3E54530E706884189428A4322E5487040
:1009AD0003020A0D789EE6FAC3E54433F8E54533B4
:1009BD00F91129E930E70BC3E89480E994FF40135E
:1009CD0021E4C3E8947FE99400500221E4787F7913
:1009DD000021E4788079FFE820E715C3E52398F836
:1009ED004009C3E894014003020A0B7801020A0B87
:1009FD00E8F424012523F84003020A0B78FF88460A
:100A0D0022E5487003020A6F789FE6FAA842A943CF
:100A1D001129E930E70CC3E89401E994FF4016026F
:100A2D000A46C3E894FFE994005003020A4678FF92
:100A3D007900020A46780179FFE920E715C3E546FA
:100A4D0098F84009C3E894014003020A6D7800024A
:100A5D000A6DE8F424012546F84003020A6D78FF7B
:100A6D00882422020B077883E6F520120F6975E8BA
:100A7D0090E5E820ECEDA8BDA9BE120FFE756855F6
:100A8D00756900C3740013FD745513FC74552CFC6B
:100A9D0074003DFDECFAEDFBC3E89AE99B4014E5CB
:100AAD00682455F568E5693400F569EA2CFAEB3DE3
:100ABD00FB80E5AE68AF69C3E56913F9E56813F826
:100ACD00C3E913F9E813F8E56828F566E56939F522
:100ADD00677A03C3E913F9E813F8DAF7AA201A7055
:100AED0009756800756900020B071AEA6008EE289F
:100AFD00FEEF39FFDAF88E688F692275E89022785B
:100B0D0083E6FFE5E820ECF7A8BDA9BE056AC3E5BD
:100B1D006A94084052756A00E97007E56B601B0224
:100B2D000B3BC3E8956B6010E56B5006600C14022F
:100B3D000B470460F9020B47E56BF56BC394A8F8FE
:100B4D004021755CC0C3E89405F84017755C80C3FF
:100B5D00E89405F8400D755C40C3E89405F8400332
:100B6D00755C0075BB0622C3E56AB4070375BB1E31
:100B7D002230610278323062027878E52C540660BA
:100B8D001FE879A187F0A4C5F0A2F733F8C3E89563
:100B9D005C4002A85C882288248825306102885E2A
:100BAD0022788FE6FFC3EF94055018C3EF940450DD
:100BBD0020C3EF94035028C3EF94025030C3EF9439
:100BCD000150387533A075340F75353C7536058178
:100BDD00167533C075341275354075360681167528
:100BED0033707534177535D0753607811675334CDE
:100BFD0075341D7535C475360981167533287534F0
:100C0D00237535B875360B811685334F8534507580
:100C1D003B00753C0822A84FA950020C2EA849A9EB
:100C2D004A759100C3E498F594E499F5957591048E
:100C3D00D25875C820A8CCA9CD75C824AA39AB3A0D
:100C4D008839893AC3E89AF8E99BF9AA3BAB3CC3CA
:100C5D00EB13FDEA13FCC3ED13FDEC13FCC3EA9C8F
:0E0C6D00FAEB9DFBEA28FAEB39FB8A3B8B3C45
:100C7B00400122753BFF753CFF2230580281857580
:100C8B009100C3E4954BF594E4954CF5957591045F
:100C9B00D258227892E6FF7E10305B027F053063DC
:100CAB00047F037E00A93CA83B7A04C3E913F9E84F
:100CBB0013F8DAF7C3E89EF8E99400F94009C3E8A2
:100CCB009402E9940050047802E4F9E9FBE8FAC3D2
:100CDB00E913FDE813FCC3EF9403602EEF20E00D46
:100CEB00E82CF8E93DF9ECFAEDFB020D02E828F8E7
:100CFB00E939F97A02E4FBC3EF9403400D8A4D8B7B
:100D0B004E8849894A8C4B8D4C22884D894E8A4995
:100D1B008B4A8C4B8D4C22305802A122759100C30B
:100D2B00E4953BF594E4953CF595759104D25822E6
:100D3B00753E00752000020D4A753E00752040D2AD
:100D4B00AF053E20580122759D00E53CC313C3132C
:100D5B00F8086030306A06C313C313F808C3E8946D
:100D6B000A4002780A306D08C3E894044002780404
:100D7B00C3E53C9408400D759D02C3E53C941040BF
:100D8B0003759D03205803D2AF22791E206D027983
:100D9B000AD2AF0000C2AF205A0A793C206D02790B
:100DAB0014306FE03063027978C3E58B99206302CE
:100DBB0040F740D0E59BF45440B52002A14AD8C47B
:100DCB00D2AF22C25B789CE6146007E53E1470023A
:100DDB00D25B30630B0538205810753800020DF5C7
:100DEB002058071581158102175422759100C3E411
:100DFB00954DF594E4954EF595759104D25822AE28
:100E0B0025305B4F78A3E6FFBF010BD25C75250045
:100E1B00C2B1C287C281918A305C037525003058FC
:100E2B0002C123BF020BD25C752500C2B1C287C2BF
:100E3B008178A2B6010D918A305C0375250030587C
:100E4B0002C143BF030BD25C752500C2B1C287C27E
:100E5B0081B1F6305C03752500305802C15E305B02
:100E6B0004C25C8E2522C2AFC286206A03020E909A
:100E7B00900360306E0F207502C280307502C28203
:100E8B007406D5E0FD207502D282307502D28075D2
:100E9B009F02753D02D2AF22C2AF206A03020EC57C
:100EAB00900317306E17C286207502C28030750210
:100EBB00C2827406D5E0FD020EC89001FA207502BD
:100ECB00C281307502C2B1305A06E5256002D28765
:100EDB00207503759F03307503759F01753D03D214
:100EEB00AF22C2AF207502C282307502C280206A67
:100EFB0003020F0C9002D6306E07C2867406D5E043
:100F0B00FD207502D280307502D282207503759F49
:100F1B0001307503759F03753D04D2AF22C2AF201C
:100F2B006A03020F4A900295306E17207502C28237
:100F3B00307502C280C2867406D5E0FD020F4D905B
:100F4B0001E8C287305A0EE525600A207502D2B13E
:100F5B00307502D281759F02753D05D2AF22C2AFAB
:100F6B00207502C280307502C282206A03020F9084
:100F7B0090024C306E0F207502C282307502C28017
:100F8B007406D5E0FDD286207503759F033075037B
:100F9B00759F01753D06D2AF22C2AF206A03020FC7
:100FAB00CE9003B9306E1F207502C282307502C21B
:100FBB0080207502C280307502C2827406D5E0FDB6
:100FCB00020FD190020C207502C2B1307502C281A2
:100FDB00305A0EE525600A207502D281307502D297
:100FEB00B1207503759F01307503759F03753D0126
:100FFB00D2AF229001E6C2B1C287C281C282C28641
:10100B00C28022C3E54F9535E550953650012278C5
:10101B0090E6FFC3EF94055018C3EF9404501BC325
:10102B00EF9403501EC3EF94025021C3EF94015071
:10103B0024C3E54F943CF8021069C3E54F9428F89C
:10104B00021069C3E54F941AF8021069C3E54F9477
:10105B0012F8021069C3E54F940AF8021069E550C3
:0F106B009400F9884F89502230580302107322E5
:10107A00788476037885760478867609788F76037D
:10108A00789076057895760278927603789B760D35
:10109A007893760578877604789C76017888760145
:1010AA007889760178827604788C7601788D760054
:1010BA00788E76B478967625789776D078987678FA
:1010CA00789976C8789A7604789D7600227893E69D
:1010DA00FF756409756501C3BF0209756405756505
:1010EA000102111CC3BF030975640575650202116B
:1010FA001CC3BF040975640575650302111CC3BFCF
:10110A000506756409756507C3BF0606756400752B
:10111A0065007887E6FFC26CC3BF0302D26CC26B5C
:10112A00C3BF0402D26BC26A7418552D6002D26A18
:10113A00C26E6002D26ED26F6002C26FC2757888C8
:10114A00E630E102D275C2767889E630E102D276DB
:10115A00C3EF94026008758E01D26D02116D758E0F
:10116A0000C26D227880E61490008093789EF6780B
:10117A0081E61490008093789FF6120FFE22789BE6
:10118A00E61490008D9378A0F6120FFE227886E678
:10119A001490009A9378A1F6120FFE22789CE61416
:1011AA009000A79378A2F6789CE6149000AC937806
:1011BA00A3F6120FFE22C2B3789DE66002D2B322D2
:1011CA007896E6FA7897E6FB3077047A007BFFC3D5
:1011DA00EB9AFCC3948250027C82756C00056CEC1D
:1011EA00856CF0A4C3E5F0948040F222C2D353D9AF
:1011FA00BF7581C043FF8012075E75EF0243B203D9
:10120A00E5B324044002F5B375803875A4C775F1B7
:10121A00FF75D4DF7590FF75A50075F20075D500CE
:10122A0075A0FF75A60075F30075D60075B0E47554
:10123A00A71B75F4FF75E241120FFEE4F8F6D8FD1C
:10124A00117A12178411D7316E3188319731A6314C
:10125A00C031CA7898866D120FFE7588507589025A
:10126A0075C82475910475D8401207721207811245
:10127A00076A12078812076A12078F12076A121C76
:10128A00CD12077212077212076E75A82275B8027C
:10129A0075E69075F610759B80759D0375D10E7570
:1012AA00BC5875BB0675BA1F75E88012075ED2AFC7
:1012BA00120A7043DA01C2D8C26912077275300184
:1012CA00D2597A05E55770027A05120762E558C3C2
:1012DA00940240EEE52E541F855A59F55AB559E243
:1012EA00DAE2C25953DACF20760343DA20307603A2
:1012FA0043DA10C2D8C26912076E12076278027402
:10130A001F552E70027800C3E5589840EDC2AF12FF
:10131A000781120781120781D2AF1207727547003F
:10132A00120762788CE6C3940150030213F3E53086
:10133A00C3940150030213F3741F552E6035C3E59D
:10134A005894FF50030213F3C2AF120796D2AF129A
:10135A00076EC3E558940150EFC2AF120781120716
:10136A0066120781D2AF12076EC3E55894FF40E9AF
:10137A00021D527F05D27731CA12076EC2AFC277F9
:10138A0031CAC3E558947FD2AF4068C2AF120796FC
:10139A00D2AFDFE1C3E55894057897F612077212C7
:1013AA001820121CD57F0AD27731CA12076EC2AF33
:1013BA00C27731CAC3E558947FD2AF50E8C2AF12A0
:1013CA000781120766120781D2AFDFDBE5582405D1
:1013DA007896F6120772121820121D0412076EC3AD
:1013EA00E55894FF40F6021D52C3E558954740035D
:1013FA0085584712076EC3E55894014002612AC214
:10140A00AF120796120796120796D2AF1207727595
:10141A003000E4F531F5320531E531F47036053244
:10142A00789AE67828146012785014600D78A0141F
:10143A00600878F0146003753200C3E532984014EE
:10144A0015327899866DC2AF120796D2AF78988610
:10145A006D12076E120762E5287008741F552E7008
:0F146A000241CAC3E558940640AD12076EE5284B
:1014790070030212CA120FFEE4F522F523F524F5D2
:1014890025755CFF7885865FF53FF540F541F542A6
:10149900F543F56AF548F52BF52CF55B120BAE759E
:1014A9006A0875BB1E12075E120B08E5E820ECFB03
:1014B900A8BDA9BEE97001F8886B120B0C756A0802
:1014C90075BB1E7895E630E0030215117887E6FEB4
:1014D900760211D77887EEF6D261C2AF120B7E85FC
:1014E900225C85225DD2AFC26175250075620075E7
:1014F9006301D260D263753800120F69120FA4120A
:101509000C2A120BAE02163A7887E6FE7603789318
:10151900E6FD760511D77887EEF67893EDF6D26079
:10152900D261D26E120F69120FA4120B7E12075EDE
:10153900120E7112075E12075E120EA312076212D3
:101549000EED120762120762120F28120766120FB8
:101559006912076212075EC261D262120B08120B8E
:101569000C120B7E756A0875BB1E120FA4120C2390
:10157900120C9E110E1173120E71120C23120C9E75
:10158900110E1173120EA3120C23120C9E110E11BF
:1015990073120EED120C23120C9E110E1173120F01
:1015A90028120C23120C9E110E1173120F69120CC2
:1015B90023120C9E110EC3E54F9535E55095364023
:1015C9000C1173C3E558940150910217541173C259
:1015D900627887E6FE760211D77887EEF685225C77
:1015E900855E5D855E25756200756301D263753818
:1015F90000C2AF207502C282307502C28020750216
:10160900C280307502C282742DD5E0FDD2AF120FAF
:10161900A4120C2A120C85120C9E120D22756A0056
:1016290075BB0602163A11D7120FA4756A0075BB6D
:1016390006120D44120DCE120DF6120880120E0A72
:10164900120E71120C2A120C85120C9E120D221206
:101659000D3B120DCE120DF612090D120E0A120EC5
:10166900A3120C2A120C85120C9E120D22120D4483
:10167900120DCE120DF612094D120E0A120EED12AE
:101689000C2A120C85120C9E120D22120D3B120D02
:10169900CE120DF61209AA120E0A120F28120C2ADE
:1016A900120C85120C9E120D22120D44120DCE122F
:1016B9000DF6120A0E120E0A120F69120C2A120CDA
:1016C90085120C9E120D22120D3B120B08120DCE23
:1016D900120DF6120B0C120E0A120FA4120C2A127A
:1016E9000C85120C9E120D2230632A755CFF755D04
:1016F900FF756200756301C3E5389464400AC263EB
:10170900D26475371402171EC3E5589401400302C9
:10171900163A021754306419E537147005C2640289
:10172900162FF537C3E5589401400302163A0217FC
:1017390054C3E55B94825013741F552E7004E52839
:101749006009C3E53C94F05002C13A120FFE788754
:10175900E6FE760211D77887EEF6E4F522F523F551
:1017690024F525F55FC26012075E120FFE741F553E
:101779002E7006E528700241CA811C901A0D782046
:10178900121C00E520B45A0CA3121C00E520B4A5D4
:10179900030217A5117A12182002181F78827604FD
:1017A900901A077884121C00A308121C00A30812BF
:1017B9001C00A308121C00A308121C00A308121C79
:1017C90000A308A308A308121C00A308A308A308E0
:1017D900121C00A308121C00A308A308121C00A3D2
:1017E90008121C00A308A308121C00A308121C005D
:1017F900A308121C00A308121C00A308121C00A3B2
:1018090008121C00A308121C00A308121C00A3083C
:10181900121C00901A2122C2AF121C3F121C1990EF
:101829001A00740A121C05A37404121C05A374106F
:10183900121C05901A077884121C04A308121C04B0
:10184900A308121C04A308121C04A308121C04A355
:1018590008121C04A308A308A308121C04A308A3C4
:0F18690008A308121C04A308121C04A308A30858
:10187800121C04A308121C04A308A308121C04A326
:1018880008121C04A308121C04A308121C04A308B1
:10189800121C04A308121C04A308121C04A3081297
:1018A8001C04A308121C04121C52121C30901A218A
:0118B800220D
:101A00000A0410FFFFFFFF0304090401015AA501A6
:101A1000FFFF0305FF0305FF0225D0FAFA040D01BD
:021A200000FFC5
:101A4000235467794B463430412320202020202026
:101A500023424C48454C4923463331302320202033
:101A60002020202020202020202020202020202076
:101C0000E493F622E6438F01538FFD75EF0275B71B
:101C1000A575B7F1F0538FFE22438F02438F0175F4
:101C2000EF0275B7A575B7F1901A0DF0538FFC222E
:101C3000901A0D745A9105901A0E74A59105227A86
:101C40003079D07820901A409100E520F709A3DA86
:101C5000F7227A3079D0901A40E7910509A3DAF992
:101C600022AB6EA86FBB01057984021CCABB0205BA
:101C70007985021CCABB03057995021CCABB040501
:101C80007986021CCABB0505798F021CCABB0605F2
:101C90007990021CCABB07057992021CCABB0805D1
:101CA000799B021CCABB09057993021CCABB0A05B1
:101CB0007987021CCABB0B05799C021CCABB0C05A8
:101CC0007988021CCA7989021CCAE8F7227C0512AD
:101CD0000772DCFB22C2AF12078112078812078F3E
:101CE00012079612076612078112078812078F12D1
:101CF000079612076612078112078812078F1207CC
:101D000096D2AF22C2AF12079612078F120788121F
:101D1000078112076612079612078F1207881207AB
:101D20008112076612079612078F12078812078121
:101D3000D2AF22AE6EAF6FC2AF120781120781120F
:101D40000781120766DEF2120796120766DFF8D2E5
:101D5000AF2291D591CD91CD756E01756F017570E2
:101D600000B1337C05AD58120772C3ED955870F57C
:101D7000C3E55894014009C3E55894FF4032A18E51
:101D8000916112182091D5C2AF75EF1291CDDCD5BB
:101D90000570C3E5709403500280C691CD056FE5D0
:101DA0006E149000B193F808C3E56F98500280AEAE
:101DB00091CD91CD056EC3E56E940E5002809C12BC
:0C1DC000107A121820C2AF75EF1291CDFE
:00000001FF
